 pvr2d_unittest

 Timestamp is 4be8ceeb (Tue May 11 12:28:43 2010)

 Preferred load address is 00010000

 Start         Length     Name                   Class
 0001:00000000 00000004H .CRT$XCA                CODE
 0001:00000004 00000004H .CRT$XCZ                CODE
 0001:00000008 00000004H .CRT$XIA                CODE
 0001:0000000c 00000004H .CRT$XIZ                CODE
 0001:00000010 00000004H .CRT$XPA                CODE
 0001:00000014 00000004H .CRT$XPZ                CODE
 0001:00000018 00000004H .CRT$XTA                CODE
 0001:0000001c 00000004H .CRT$XTZ                CODE
 0001:00000020 00000560H .rdata                  CODE
 0001:00000580 0000002bH .rdata$debug            CODE
 0001:000005ac 00002334H .text                   CODE
 0001:000028e0 0000001cH .xdata                  CODE
 0001:000028fc 00000028H .idata$2                CODE
 0001:00002924 00000014H .idata$3                CODE
 0001:00002938 00000118H .idata$4                CODE
 0001:00002a50 000001bcH .idata$6                CODE
 0001:00002c0c 00000000H .edata                  CODE
 0002:00000000 00000118H .idata$5                DATA
 0002:00000118 0000a41cH .data                   DATA
 0002:0000a534 00000010H .bss                    DATA
 0003:00000000 000000f8H .pdata                  DATA

  Address         Publics by Value              Rva+Base       Lib:Object

 0000:00000000       ___safe_se_handler_table   00000000     <absolute>
 0000:00000000       ___safe_se_handler_count   00000000     <absolute>
 0001:00000000       __xc_a                     00011000     corelib0:crt0init.obj
 0001:00000004       __xc_z                     00011004     corelib0:crt0init.obj
 0001:00000008       __xi_a                     00011008     corelib0:crt0init.obj
 0001:0000000c       __xi_z                     0001100c     corelib0:crt0init.obj
 0001:00000010       __xp_a                     00011010     corelib0:crt0init.obj
 0001:00000014       __xp_z                     00011014     corelib0:crt0init.obj
 0001:00000018       __xt_a                     00011018     corelib0:crt0init.obj
 0001:0000001c       __xt_z                     0001101c     corelib0:crt0init.obj
 0001:0000003c       ??_C@_03KDDEMCGN@car?$AA@  0001103c     pvr2d_unittest.obj
 0001:00000040       car                        00011040     pvr2d_unittest.obj
 0001:00000064       ??_C@_0BK@HIALDAHE@PowerVR?5device?5not?5found?6?$AA@ 00011064     pvr2d_unittest.obj
 0001:00000080       ??_C@_0BN@GFNHPLBJ@AllocAndLoadPVR2DBmp?5failed?6?$AA@ 00011080     pvr2d_unittest.obj
 0001:000000a0       ??_C@_0BB@PMCMFBOJ@PVR2DBlt?5failed?6?$AA@ 000110a0     pvr2d_unittest.obj
 0001:000000b4       ??_C@_0BL@JHCEAGAF@PVR2DGetScreenMode?5failed?6?$AA@ 000110b4     pvr2d_unittest.obj
 0001:000000d0       ??_C@_0BM@BHLBHGAL@PVR2DGetFrameBuffer?5failed?6?$AA@ 000110d0     pvr2d_unittest.obj
 0001:000000ec       ??_C@_0CB@EIKIBEIE@PVR2DCreateDeviceContext?5failed?6@ 000110ec     pvr2d_unittest.obj
 0001:00000110       ??_C@_0BO@DCKNHKCE@PVR2DEnumerateDevices?5failed?6?$AA@ 00011110     pvr2d_unittest.obj
 0001:00000130       ??_C@_0P@LEGHBOFO@malloc?5failed?6?$AA@ 00011130     pvr2d_unittest.obj
 0001:00000140       ??_C@_0CH@BKOEDJLC@Warning?5?9?5PVR2D?5API?5revision?5mis@ 00011140     pvr2d_unittest.obj
 0001:00000168       ??_C@_1BI@FPJLJJJA@?$AAD?$AAu?$AAm?$AAm?$AAy?$AAW?$AAi?$AAn?$AAd?$AAo?$AAw?$AA?$AA@ 00011168     wince_unittests.obj
 0001:00000180       ??_C@_1KE@BDGMONOJ@?$AAH?$AA?3?$AA?2?$AAW?$AAI?$AAN?$AAC?$AAE?$AA6?$AA0?$AA0?$AA?2?$AAP?$AAL?$AAA?$AAT?$AAF?$AAO?$AAR?$AAM?$AA?2?$AAS?$AAM?$AAD?$AAK?$AAV?$AA2?$AA1?$AA0?$AA?2?$AAS?$AAR@ 00011180     wince_unittests.obj
 0001:00000224       ??_C@_1CI@OHCJFJPM@?$AAE?$AAR?$AAR?$AAO?$AAR?$AA?3?$AA?5?$AA?$CF?$AAs?$AA?5?$AAl?$AAi?$AAn?$AAe?$AA?5?$AA?$CF?$AAd?$AA?3?$AA?5?$AA?$AA@ 00011224     wince_unittests.obj
 0001:0000024c       ??_C@_1CK@MPGKAOE@?$AA?$CI?$AAe?$AAr?$AAr?$AAo?$AAr?$AA?5?$AAc?$AAo?$AAd?$AAe?$AA?3?$AA?5?$AA?$CF?$AAd?$AA?$CJ?$AA?3?$AA?5?$AA?$CF?$AAs?$AA?$AA@ 0001124c     wince_unittests.obj
 0001:00000278       ??_C@_1M@DMCDIEDK@?$AAP?$AAK?$AAM?$AA1?$AA?3?$AA?$AA@ 00011278     wince_unittests.obj
 0001:00000284       ??_C@_0L@GPAGIAIC@?9disablepm?$AA@ 00011284     wince_unittests.obj
 0001:00000290       ??_C@_1M@ILHOPKA@?$AAE?$AAr?$AAr?$AAo?$AAr?$AA?$AA@ 00011290     wince_unittests.obj
 0001:0000029c       ??_C@_1DG@PCJNAHOH@?$AAF?$AAa?$AAi?$AAl?$AAe?$AAd?$AA?5?$AAt?$AAo?$AA?5?$AAg?$AAe?$AAt?$AA?5?$AAm?$AAo?$AAn?$AAi?$AAt?$AAo?$AAr?$AA?5?$AAi?$AAn?$AAf?$AAo?$AA?$AA@ 0001129c     wince_unittests.obj
 0001:000002d4       ??_C@_07FBLHGNAH@app?4exe?$AA@ 000112d4     wince_unittests.obj
 0001:0000068c       main                       0001168c f   pvr2d_unittest.obj
 0001:0000092c       DummyWndProc               0001192c f   wince_unittests.obj
 0001:00000998       ForceDesktopRedraw         00011998 f   wince_unittests.obj
 0001:00000a80       WinMain                    00011a80 f   wince_unittests.obj
 0001:00000d28       PVR2DMemAlloc              00011d28 f   libpvr2d:pvr2dmem.obj
 0001:00000de4       PVR2DMemFree               00011de4 f   libpvr2d:pvr2dmem.obj
 0001:00000eb0       PVR2DEnumerateDevices      00011eb0 f   libpvr2d:pvr2dinit.obj
 0001:00001280       PVR2DCreateDeviceContext   00012280 f   libpvr2d:pvr2dinit.obj
 0001:000014a8       PVR2DDestroyDeviceContext  000124a8 f   libpvr2d:pvr2dinit.obj
 0001:000015ac       PVR2DGetAPIRev             000125ac f   libpvr2d:pvr2dinit.obj
 0001:000015d0       GetPvrSrvPixelFormat       000125d0 f   libpvr2d:pvr2dblt.obj
 0001:00001640       PVR2DQueryBlitsComplete    00012640 f   libpvr2d:pvr2dblt.obj
 0001:00001f5c       PVR2DBlt                   00012f5c f   libpvr2d:pvr2dblt.obj
 0001:00001f68       PVR2DGetFrameBuffer        00012f68 f   libpvr2d:pvr2dmode.obj
 0001:00001fa4       PVR2DGetScreenMode         00012fa4 f   libpvr2d:pvr2dmode.obj
 0001:00002080       DestroyFlipChain           00013080 f   libpvr2d:pvr2dflip.obj
 0001:00002150       DefWindowProcW             00013150 f   coredll:COREDLL.dll
 0001:00002160       EndPaint                   00013160 f   coredll:COREDLL.dll
 0001:00002170       BeginPaint                 00013170 f   coredll:COREDLL.dll
 0001:00002180       DestroyWindow              00013180 f   coredll:COREDLL.dll
 0001:00002190       UpdateWindow               00013190 f   coredll:COREDLL.dll
 0001:000021a0       ShowWindow                 000131a0 f   coredll:COREDLL.dll
 0001:000021b0       CreateWindowExW            000131b0 f   coredll:COREDLL.dll
 0001:000021c0       GetSystemMetrics           000131c0 f   coredll:COREDLL.dll
 0001:000021d0       RegisterClassW             000131d0 f   coredll:COREDLL.dll
 0001:000021e0       GetModuleHandleW           000131e0 f   coredll:COREDLL.dll
 0001:000021f0       ReleasePowerRequirement    000131f0 f   coredll:COREDLL.dll
 0001:00002200       NKDbgPrintfW               00013200 f   coredll:COREDLL.dll
 0001:00002210       FormatMessageW             00013210 f   coredll:COREDLL.dll
 0001:00002220       GetLastError               00013220 f   coredll:COREDLL.dll
 0001:00002230       SetPowerRequirement        00013230 f   coredll:COREDLL.dll
 0001:00002240       WideCharToMultiByte        00013240 f   coredll:COREDLL.dll
 0001:00002250       SetCursorPos               00013250 f   coredll:COREDLL.dll
 0001:00002260       GetCursorPos               00013260 f   coredll:COREDLL.dll
 0001:00002270       MessageBoxW                00013270 f   coredll:COREDLL.dll
 0001:00002280       GetMonitorInfo             00013280 f   coredll:COREDLL.dll
 0001:00002290       MonitorFromPoint           00013290 f   coredll:COREDLL.dll
 0001:00002320       WinMainCRTStartup          00013320 f   corelib0:pegwmain.obj
 0001:00002354       __GSHandlerCheckCommon     00013354 f   corelib0:gshandler.obj
 0001:00002390       __GSHandlerCheck           00013390 f   corelib0:gshandler.obj
 0001:000023b4       __security_init_cookie     000133b4 f   corelib0:seccinit.obj
 0001:00002410       __security_check_cookie    00013410 f   corelib0:armsecgs.obj
 0001:00002424       __gsfailure                00013424 f   corelib0:armsecgs.obj
 0001:00002530       exit                       00013530 f   corelib0:cexit.obj
 0001:00002548       _exit                      00013548 f   corelib0:cexit.obj
 0001:00002588       _initterm                  00013588 f   corelib0:crt0dat.obj
 0001:000025bc       _cinit                     000135bc f   corelib0:crt0dat.obj
 0001:000025f0       free                       000135f0 f   corelib1:COREDLL.dll
 0001:00002600       calloc                     00013600 f   corelib1:COREDLL.dll
 0001:00002610       malloc                     00013610 f   corelib1:COREDLL.dll
 0001:00002620       printf                     00013620 f   corelib1:COREDLL.dll
 0001:00002630       memset                     00013630 f   corelib1:COREDLL.dll
 0001:00002640       _stricmp                   00013640 f   corelib1:COREDLL.dll
 0001:00002650       _isctype                   00013650 f   corelib1:COREDLL.dll
 0001:00002660       wcslen                     00013660 f   corelib1:COREDLL.dll
 0001:00002670       _XcptFilter                00013670 f   corelib1:COREDLL.dll
 0001:00002680       __C_specific_handler       00013680 f   corelib1:COREDLL.dll
 0001:00002690       __security_gen_cookie2     00013690 f   corelib1:COREDLL.dll
 0001:000026a0       __report_gsfailure         000136a0 f   corelib1:COREDLL.dll
 0001:000026b0       PVRSRVFreeUserModeMem      000136b0 f   srvclum:SRVCLUM.dll
 0001:000026c0       PVRSRVAllocDeviceMem       000136c0 f   srvclum:SRVCLUM.dll
 0001:000026d0       PVRSRVCallocUserModeMem    000136d0 f   srvclum:SRVCLUM.dll
 0001:000026e0       PVRSRVMemSet               000136e0 f   srvclum:SRVCLUM.dll
 0001:000026f0       PVRSRVFreeDeviceMem        000136f0 f   srvclum:SRVCLUM.dll
 0001:00002700       PVRSRVUnwrapExtMemory      00013700 f   srvclum:SRVCLUM.dll
 0001:00002710       PVRSRVUnmapDeviceMemory    00013710 f   srvclum:SRVCLUM.dll
 0001:00002720       PVRSRVDisconnect           00013720 f   srvclum:SRVCLUM.dll
 0001:00002730       PVRSRVCloseDCDevice        00013730 f   srvclum:SRVCLUM.dll
 0001:00002740       PVRSRVMemCopy              00013740 f   srvclum:SRVCLUM.dll
 0001:00002750       PVRSRVGetDCInfo            00013750 f   srvclum:SRVCLUM.dll
 0001:00002760       PVRSRVOpenDCDevice         00013760 f   srvclum:SRVCLUM.dll
 0001:00002770       PVRSRVAcquireDeviceData    00013770 f   srvclum:SRVCLUM.dll
 0001:00002780       PVRSRVEnumerateDevices     00013780 f   srvclum:SRVCLUM.dll
 0001:00002790       PVRSRVEnumerateDeviceClass 00013790 f   srvclum:SRVCLUM.dll
 0001:000027a0       PVRSRVConnect              000137a0 f   srvclum:SRVCLUM.dll
 0001:000027b0       PVRSRVUnmapDeviceClassMemory 000137b0 f   srvclum:SRVCLUM.dll
 0001:000027c0       PVRSRVMapDeviceClassMemory 000137c0 f   srvclum:SRVCLUM.dll
 0001:000027d0       PVRSRVGetDCSystemBuffer    000137d0 f   srvclum:SRVCLUM.dll
 0001:000027e0       PVRSRVEnumDCDims           000137e0 f   srvclum:SRVCLUM.dll
 0001:000027f0       PVRSRVAllocUserModeMem     000137f0 f   srvclum:SRVCLUM.dll
 0001:00002800       PVRSRVEnumDCFormats        00013800 f   srvclum:SRVCLUM.dll
 0001:00002810       PVRSRVDestroyDeviceMemContext 00013810 f   srvclum:SRVCLUM.dll
 0001:00002820       PVRSRVReleaseMiscInfo      00013820 f   srvclum:SRVCLUM.dll
 0001:00002830       SGXDestroyTransferContext  00013830 f   srvclum:SRVCLUM.dll
 0001:00002840       SGXCreateTransferContext   00013840 f   srvclum:SRVCLUM.dll
 0001:00002850       PVRSRVCreateDeviceMemContext 00013850 f   srvclum:SRVCLUM.dll
 0001:00002860       PVRSRVGetMiscInfo          00013860 f   srvclum:SRVCLUM.dll
 0001:00002870       PVRSRVEventObjectWait      00013870 f   srvclum:SRVCLUM.dll
 0001:00002880       SGX2DQueryBlitsComplete    00013880 f   srvclum:SRVCLUM.dll
 0001:00002890       PVRSRVClockus              00013890 f   srvclum:SRVCLUM.dll
 0001:000028a0       SGXQueueTransfer           000138a0 f   srvclum:SRVCLUM.dll
 0001:000028b0       PVRSRVDestroyDCSwapChain   000138b0 f   srvclum:SRVCLUM.dll
 0001:000028c0       PVRSRVSwapToDCSystem       000138c0 f   srvclum:SRVCLUM.dll
 0001:000028d0       TerminateProcess           000138d0 f   coredll:COREDLL.dll
 0001:000028fc       __IMPORT_DESCRIPTOR_COREDLL 000138fc     coredll:COREDLL.dll
 0001:00002910       __IMPORT_DESCRIPTOR_SRVCLUM 00013910     srvclum:SRVCLUM.dll
 0001:00002924       __NULL_IMPORT_DESCRIPTOR   00013924     coredll:COREDLL.dll
 0002:00000000       __imp_DefWindowProcW       00014000     coredll:COREDLL.dll
 0002:00000004       __imp_EndPaint             00014004     coredll:COREDLL.dll
 0002:00000008       __imp_BeginPaint           00014008     coredll:COREDLL.dll
 0002:0000000c       __imp_DestroyWindow        0001400c     coredll:COREDLL.dll
 0002:00000010       __imp_UpdateWindow         00014010     coredll:COREDLL.dll
 0002:00000014       __imp_ShowWindow           00014014     coredll:COREDLL.dll
 0002:00000018       __imp_CreateWindowExW      00014018     coredll:COREDLL.dll
 0002:0000001c       __imp_GetSystemMetrics     0001401c     coredll:COREDLL.dll
 0002:00000020       __imp_RegisterClassW       00014020     coredll:COREDLL.dll
 0002:00000024       __imp_GetModuleHandleW     00014024     coredll:COREDLL.dll
 0002:00000028       __imp_ReleasePowerRequirement 00014028     coredll:COREDLL.dll
 0002:0000002c       __imp_NKDbgPrintfW         0001402c     coredll:COREDLL.dll
 0002:00000030       __imp_FormatMessageW       00014030     coredll:COREDLL.dll
 0002:00000034       __imp_GetLastError         00014034     coredll:COREDLL.dll
 0002:00000038       __imp_SetPowerRequirement  00014038     coredll:COREDLL.dll
 0002:0000003c       __imp_WideCharToMultiByte  0001403c     coredll:COREDLL.dll
 0002:00000040       __imp_SetCursorPos         00014040     coredll:COREDLL.dll
 0002:00000044       __imp_GetCursorPos         00014044     coredll:COREDLL.dll
 0002:00000048       __imp_MessageBoxW          00014048     coredll:COREDLL.dll
 0002:0000004c       __imp_GetMonitorInfo       0001404c     coredll:COREDLL.dll
 0002:00000050       __imp_MonitorFromPoint     00014050     coredll:COREDLL.dll
 0002:00000054       __imp_free                 00014054     corelib1:COREDLL.dll
 0002:00000058       __imp_calloc               00014058     corelib1:COREDLL.dll
 0002:0000005c       __imp_malloc               0001405c     corelib1:COREDLL.dll
 0002:00000060       __imp_printf               00014060     corelib1:COREDLL.dll
 0002:00000064       __imp_memset               00014064     corelib1:COREDLL.dll
 0002:00000068       __imp__stricmp             00014068     corelib1:COREDLL.dll
 0002:0000006c       __imp__isctype             0001406c     corelib1:COREDLL.dll
 0002:00000070       __imp_wcslen               00014070     corelib1:COREDLL.dll
 0002:00000074       __imp__XcptFilter          00014074     corelib1:COREDLL.dll
 0002:00000078       __imp___C_specific_handler 00014078     corelib1:COREDLL.dll
 0002:0000007c       __imp___security_gen_cookie2 0001407c     corelib1:COREDLL.dll
 0002:00000080       __imp___report_gsfailure   00014080     corelib1:COREDLL.dll
 0002:00000084       __imp_TerminateProcess     00014084     coredll:COREDLL.dll
 0002:00000088       \177COREDLL_NULL_THUNK_DATA 00014088     coredll:COREDLL.dll
 0002:0000008c       __imp_PVRSRVAllocDeviceMem 0001408c     srvclum:SRVCLUM.dll
 0002:00000090       __imp_PVRSRVFreeUserModeMem 00014090     srvclum:SRVCLUM.dll
 0002:00000094       __imp_PVRSRVMemSet         00014094     srvclum:SRVCLUM.dll
 0002:00000098       __imp_PVRSRVFreeDeviceMem  00014098     srvclum:SRVCLUM.dll
 0002:0000009c       __imp_PVRSRVUnwrapExtMemory 0001409c     srvclum:SRVCLUM.dll
 0002:000000a0       __imp_PVRSRVUnmapDeviceMemory 000140a0     srvclum:SRVCLUM.dll
 0002:000000a4       __imp_PVRSRVDisconnect     000140a4     srvclum:SRVCLUM.dll
 0002:000000a8       __imp_PVRSRVCloseDCDevice  000140a8     srvclum:SRVCLUM.dll
 0002:000000ac       __imp_PVRSRVMemCopy        000140ac     srvclum:SRVCLUM.dll
 0002:000000b0       __imp_PVRSRVGetDCInfo      000140b0     srvclum:SRVCLUM.dll
 0002:000000b4       __imp_PVRSRVOpenDCDevice   000140b4     srvclum:SRVCLUM.dll
 0002:000000b8       __imp_PVRSRVAcquireDeviceData 000140b8     srvclum:SRVCLUM.dll
 0002:000000bc       __imp_PVRSRVEnumerateDevices 000140bc     srvclum:SRVCLUM.dll
 0002:000000c0       __imp_PVRSRVEnumerateDeviceClass 000140c0     srvclum:SRVCLUM.dll
 0002:000000c4       __imp_PVRSRVConnect        000140c4     srvclum:SRVCLUM.dll
 0002:000000c8       __imp_PVRSRVUnmapDeviceClassMemory 000140c8     srvclum:SRVCLUM.dll
 0002:000000cc       __imp_PVRSRVMapDeviceClassMemory 000140cc     srvclum:SRVCLUM.dll
 0002:000000d0       __imp_PVRSRVGetDCSystemBuffer 000140d0     srvclum:SRVCLUM.dll
 0002:000000d4       __imp_PVRSRVEnumDCDims     000140d4     srvclum:SRVCLUM.dll
 0002:000000d8       __imp_PVRSRVAllocUserModeMem 000140d8     srvclum:SRVCLUM.dll
 0002:000000dc       __imp_PVRSRVEnumDCFormats  000140dc     srvclum:SRVCLUM.dll
 0002:000000e0       __imp_PVRSRVDestroyDeviceMemContext 000140e0     srvclum:SRVCLUM.dll
 0002:000000e4       __imp_PVRSRVReleaseMiscInfo 000140e4     srvclum:SRVCLUM.dll
 0002:000000e8       __imp_SGXDestroyTransferContext 000140e8     srvclum:SRVCLUM.dll
 0002:000000ec       __imp_SGXCreateTransferContext 000140ec     srvclum:SRVCLUM.dll
 0002:000000f0       __imp_PVRSRVCreateDeviceMemContext 000140f0     srvclum:SRVCLUM.dll
 0002:000000f4       __imp_PVRSRVGetMiscInfo    000140f4     srvclum:SRVCLUM.dll
 0002:000000f8       __imp_PVRSRVEventObjectWait 000140f8     srvclum:SRVCLUM.dll
 0002:000000fc       __imp_SGX2DQueryBlitsComplete 000140fc     srvclum:SRVCLUM.dll
 0002:00000100       __imp_PVRSRVClockus        00014100     srvclum:SRVCLUM.dll
 0002:00000104       __imp_SGXQueueTransfer     00014104     srvclum:SRVCLUM.dll
 0002:00000108       __imp_PVRSRVDestroyDCSwapChain 00014108     srvclum:SRVCLUM.dll
 0002:0000010c       __imp_PVRSRVSwapToDCSystem 0001410c     srvclum:SRVCLUM.dll
 0002:00000110       __imp_PVRSRVCallocUserModeMem 00014110     srvclum:SRVCLUM.dll
 0002:00000114       \177SRVCLUM_NULL_THUNK_DATA 00014114     srvclum:SRVCLUM.dll
 0002:00000118       car_data                   00014118     pvr2d_unittest.obj
 0002:0000a52c       __security_cookie          0001e52c     corelib0:seccinit.obj
 0002:0000a530       __security_cookie_complement 0001e530     corelib0:seccinit.obj
 0002:0000a534       pfnRegisteredWndProc       0001e534     wince_unittests.obj
 0002:0000a538       _exitflag                  0001e538     corelib0:cexit.obj
 0002:0000a53c       __onexitend                0001e53c     <common>
 0002:0000a540       __onexitbegin              0001e540     <common>

 entry point at        0001:00002320

 Static symbols

 0001:000005ac       AllocAndLoadPVR2DBmp       000115ac f   pvr2d_unittest.obj
 0001:00001098       InitDisplayDevice          00012098 f   libpvr2d:pvr2dinit.obj
 0001:0000171c       AltBltClipped              0001271c f   libpvr2d:pvr2dblt.obj
 0001:000022a8       WinMainCRTStartupHelper    000132a8 f   corelib0:pegwmain.obj
 0001:00002468       doexit                     00013468 f   corelib0:cexit.obj
